:020000040000fa
:08000000007d04000100000076
:020000040000fa
:1002000000000000000000000000000000000000ee
:1002100000000000000000000000000000000000de
:1002200000000000000000000000000000000000ce
:1002300000000000000000000000000000000000be
:020000040002f8
:10fa0000701680000040a700000104000000000004
:10fa10000f8820008079220000018800000000008b
:10fa20004440a80020002000a00188000000000041
:10fa30002601070000422800601088000e22ef0017
:10fa40001221ef008ce0a9000ea1ef0000002800b9
:10fa5000900888004221ef004221a8008420a900dc
:10fa60008c20a900400020005e0007000a21ef0062
:10fa70005c0007000000e900fdff3a0013e1a90067
:10fa8000500880000004b0004780de000000e9005c
:10fa9000a01088000ca2a9000f42a8001f00370088
:10faa0000e02ae00feff3700901080006f04e100f0
:10fab0004220af0000010400000000006104e100ea
:10fac0000a0032006204e100190032006304e10020
:10fad0000100320013003700100020008010880061
:10fae00010002000801088000c003700490007003b
:10faf00090018800470007000080fd0045000700d6
:10fb00009080ba00811088009000ba000180fd004a
:10fb1000811088000180fd008110880050052000c0
:10fb200001003700f00f200080108800dcff370054
:10fb30000002eb003700070090018800203b88009e
:10fb40003400070063e7b7003200070062e7b70040
:10fb50003000070080017800028020002d0007009f
:10fb6000005978008301e900fcff3a000404e0003a
:10fb7000ecff3a0002802000153b8000800f20003f
:10fb80003240e30003003a00880024001300200004
:10fb90000b003700f00720003240e30004003a0079
:10fba00050072400580024000302200003003700ff
:10fbb000100724001800240003042000220007007e
:10fbc000b20abb008301e90003003200b29abb0015
:10fbd0008301e900faff3a00080078001a000700e4
:10fbe000ceff3700a20520008080eb008420af000c
:10fbf000060037008100e900fcff3a000201e9003d
:10fc0000f9ff3a0000010400000000008420a90070
:10fc100000000600faff2f008085eb000e02af0007
:10fc2000060037008b05e900fcff3a000a05e900f1
:10fc3000f9ff3a000f882000baff370012c2bf0058
:10fc40000042420000000600003b880050052000f2
:10fc5000303b8800a00a2000303b880061e7a80004
:10fc6000000000000000000061e7af00feff370069
:10fc7000000006000200fa00000f78000000eb0010
:10fc8000c00888001e0078000100200082002000cb
:10fc90000202b8000001eb000283b9000501780000
:10fca00006014100830020000388b90000014100e3
:10fcb00082027800e408880086c0a90021e1a8003b
:10fcc00086c0bf000080fb004600de000080fb0015
:10fcd000610060000000e000f9ff320021e1a900ae
:10fce0000080fa00000006000400fa00000f78000f
:10fcf0000000eb00100798001e0090009e0f5000bf
:10fd000006003100803e2000daff07001e00900050
:10fd10000000e80010079800f7ff37000080fa00a5
:10fd2000000006000200fa00004f7800b1168000c3
:10fd3000f00f2000008160001e80fb00c800dd0085
:10fd400000f02f000080600000007100b0168800f5
:10fd500010002000c7ff0700d6a2a8001000200056
:10fd6000c4ff0700d6a2a90010002000deff070094
:10fd70000080fa00000006000200fa00004f780040
:10fd8000d6e2a90000c8b3001e407000e5ff0700de
:10fd9000d6e2a80020002000d3ff07000080fa0070
:10fda000000006000000fa00e00124006016880050
:10fdb0000000eb00701688001000200090168800ec
:10fdc0000000eb00a0168800cfa2a800d6e2a90090
:10fdd000d6c2a900f0002000c3ff070080c3b30013
:10fde000d0ff070050002000bfff070080c3b30012
:10fdf000ccff070010002000bbff070080c3b3004a
:10fe0000c8ff070010002000b7ff0700c0c0b30004
:10fe1000c4ff070010002000b3ff070010c0b300ac
:10fe2000c0ff070020002000afff070060c0b30044
:10fe3000bcff070010002000abff0700d6e2a800bf
:10fe40000000eb00800c88000000eb00b00c880084
:10fe5000c0122000600c8800c0122000700c8800c6
:10fe600060002000800c8800007d2000900c88003d
:10fe7000007d2000a00c880060002000b00c8800ed
:10fe8000b0d421006008880011e1a8000080fa00c9
:10fe9000000006000200fa00000f78001e00780043
:10fea0001004e000070032009e0078001140780046
:10feb0009cff07001e0078000000e800000f78009b
:10fec000f6ff37000080fa00000006000000fa008c
:10fed000b4ff0700a0f72f00eeff070000c4b30037
:10fee000a5ff0700b0f82f00eaff07000080fa0026
:04fef0000000060008
:020000040000fa
:0200000401f009
:04000000e5ff000018
:020000040000fa
:0200000401f009
:04000400ff7f00007a
:020000040000fa
:0200000401f009
:04000800ffff0000f6
:020000040000fa
:0200000401f009
:04001400ffff0000ea
:020000040000fa
:10000800fa7f0100fa7f0100fa7f0100fa7f010000
:10001800fa7f0100fa7f0100fa7f0100fa7f0100f0
:10002800fa7f0100fa7f0100fa7f0100fa7f0100e0
:10003800fa7f0100fa7f0100fa7f0100fa7f0100d0
:10004800fa7f0100fa7f0100fa7f0100fa7f0100c0
:10005800fa7f0100fa7f0100fa7f0100fa7f0100b0
:10006800fa7f0100fa7f0100fa7f0100fa7f0100a0
:10007800fa7f0100fa7f0100fa7f0100fa7f010090
:10008800fa7f0100fa7f0100fa7f0100fa7f010080
:10009800fa7f0100fa7f0100fa7f0100fa7f010070
:1000a800fa7f0100fa7f0100fa7f0100fa7f010060
:1000b800fa7f0100fa7f0100fa7f0100fa7f010050
:1000c800fa7f0100fa7f0100fa7f0100fa7f010040
:1000d800fa7f0100fa7f0100fa7f0100fa7f010030
:1000e800fa7f0100fa7f0100fa7f0100fa7f010020
:0800f800fa7f0100fa7f01000c
:020000040000fa
:10010800fa7f0100fa7f0100fa7f0100fa7f0100ff
:10011800fa7f0100fa7f0100fa7f0100fa7f0100ef
:10012800fa7f0100fa7f0100fa7f0100fa7f0100df
:10013800fa7f0100fa7f0100fa7f0100fa7f0100cf
:10014800fa7f0100fa7f0100fa7f0100fa7f0100bf
:10015800fa7f0100fa7f0100fa7f0100fa7f0100af
:10016800fa7f0100fa7f0100fa7f0100fa7f01009f
:10017800fa7f0100fa7f0100fa7f0100fa7f01008f
:10018800fa7f0100fa7f0100fa7f0100fa7f01007f
:10019800fa7f0100fa7f0100fa7f0100fa7f01006f
:1001a800fa7f0100fa7f0100fa7f0100fa7f01005f
:1001b800fa7f0100fa7f0100fa7f0100fa7f01004f
:1001c800fa7f0100fa7f0100fa7f0100fa7f01003f
:1001d800fa7f0100fa7f0100fa7f0100fa7f01002f
:1001e800fa7f0100fa7f0100fa7f0100fa7f01001f
:0801f800fa7f0100fa7f01000b
:020000040000fa
:020000040002f8
:10fef4005041000031300000302f00005458000001
:10ff040035300000302f000031330000362000006f
:10ff1400004600006c610000736800006572000018
:10ff240020730000746100007274000065640000b6
:04ff34002e0000009b
:020000040000fa
:020000040002f8
:10ff3800000800008000000002000000000000002f
:10ff480000000000000000000000000000000000a9
:10ff58000000000000000000000000000000000099
:10ff68000000000000000000000000000000000089
:10ff78000000000000000000000000000000000079
:10ff88000000000000000000000000000000000069
:10ff98000000000000000000000000000000000059
:10ffa8000000000000000000000000000000000049
:10ffb8000000000000000000000000000000000039
:10ffc8000000000000000000000000000000000029
:10ffd8000000000000000000000000000000000019
:0cffe8000000000000000000000000000d
:020000040000fa
:020000040002f8
:04fff4000000fe000b
:00000001FF
